:100000000C949C070C94B9070C94B9070C94B9078D
:100010000C94B9070C94B9070C94B9070C94B90760
:100020000C94B9070C94B9070C94362A0C94082B3D
:100030000C9400250C94B9070C94B9070C94B907DB
:100040000C94B9070C94B9070C94B9070C94B90730
:100050000C94B9070C94A4250C94B9070C94B90717
:100060000C94B9070C94B9070C94B9070C94B90710
:100070000C94B9070C94B9070C94B9070C94B90700
:100080000C94B9070C94B9070C94B9070C94B907F0
:100090000C9467230C94B9070C94B9070C94B90716
:1000A0000C94B9070C94B9070C94B907800B800B1A
:1000B000AC0BAC0B140C3F0D3F0D3F0D320CCB0CB9
:1000C000DC0CDC0C752B9C2B942C9C2B942CE82B9F
:1000D0000B2C942C622C712C2A0014001A0008009E
:1000E00015001700E20004001600070009000A00CE
:1000F000E1001D001B0006001900050000000000C3
:10010000000000000151E0002B00130012000C0061
:1001100018001C002C0033000F000E000D000B0017
:10012000E500380037003600100011000000000024
:1001300000000000025101004C001E021F022F02AD
:100140003002F300A75D2002210226022702F200FE
:100150000100220223022F003000F1000000000005
:1001600000000000010001002D02250226002500EC
:100170002400340228002E02230022002100340033
:1001800001002D0020001F001E00270000000000BD
:1001900000000000010001000100290040004100B2
:1001A000420043000100E3003D003E003F004400E8
:1001B000010049003A003B003C00450000000000FF
:1001C0000000000001000100A85D35004E00520053
:1001D0004B003102A95D35024F005100500024024E
:1001E000AA5D31004D00AE004A002E000000000064
:1001F000000000000100010003A6681E7D107E7E45
:100200005F1CB8F2470C7B744B148B7566510B8CDA
:1002100076744B14AAD60F9CBAF66E3FDD38D50221
:10022000809B826D5813A4ABB5C910A2C60A7F5D2E
:100230001991A0A3CEEB3EC9F16042E74CFB746A72
:10024000562EBFDD38D3058892A6CEFF5D38D1CFBC
:10025000EF58CB6548F03585A9B28F5EF38094974F
:100260007E7597877313B08A69D40ADEC1795936CF
:10027000DB9DD6B8156FCE3C72324588DF6CA56D1C
:10028000E87696147420DCF4FA376A2732E329BF43
:10029000C4C7069D58E7877C2E9F6E49075D23647F
:1002A00054836ECBB777F72B6E0F2E6612605565B1
:1002B000FC43B358735BE867044302DEB389A06D67
:1002C0003A2779645B0C169E66B18B870C5DF2B69B
:1002D0003D71DF42038A068DEF1DA8965CED31610A
:1002E0005CA134F68C08603307003E79951B437F90
:1002F000FEB6A6D49D7672BFADC015E83731A372A5
:1003000063521D1C5D511BE1A9ED60323EA95028CE
:10031000530659E2FCE702643921564AA540808120
:10032000D55A607B6884F1E0B1B65BDFA81D6D65CE
:1003300020C0A2B9D9BB00A6DB8B015391FEC451EA
:1003400085B0967FFD51DD1403672E751C76D36E44
:10035000DD995576E5AB23FC4AD5C6E82ECA8AB3AB
:10036000F68C6CB0E9F2E79E6941EDF16DD286D86A
:100370007ECB5D476C856A23ED204093B420C7A5F2
:10038000C9AF0315AC19E52A36DF6DC58C8007CEE1
:10039000920CD806620FDD48461A53C78A8C5D5D01
:1003A000B4A102D3A9B8F3948F3FE554D41165B238
:1003B0005E090B81E375A78981396C46F6069F2794
:1003C0003BB62D5F1D4BD47B1D617489E4E3BD9862
:1003D0001BC4513BA4FAE092F7BEF24DBBFFAD4FF8
:1003E0006D68C27940AA9B8F0C324B5F3EAB599827
:1003F000B3F51DAC5EBC78D3016C64152FD871A623
:100400002D45E12242E44E043C7DF44021B46705D1
:10041000A8E2F372874C7DD91B6597F3C2E3E4C869
:10042000D2DEF6EFDCBB44085EE2452701B0F643BE
:10043000E73AF6DC9DEDF3C50CB89C983AD836EE59
:10044000967267E78191D5050AE082D58FE8F9B009
:10045000C9CF93E704C5BC2B43567EE8677CE5FB18
:1004600049AD5E9F2513DE6E6EE9F1EC870B598175
:10047000768476B324AF30FD278BABD8008B9B0CF2
:10048000D2B24E5E9D1D96010067C15F0220FD4500
:100490006A01605845CA4721905AC443261AD7A515
:1004A0004AB25D2B3549FBA51792211E939667A290
:1004B0007E367ADE5FBE7A589DF878A3FAC8D517E3
:1004C000F021978C80B54B3BBDBB4121A85067F70D
:1004D000E71980108ECE04183F516B77D89E16AF67
:1004E000ECEF48164D9E8538183ED42887602AF6D2
:1004F0007F09866F9C3C3AFFABD061A2970D719447
:100500007EFDB98002896AB3846C2A7762BE0BF4DF
:10051000AFAC7B7C8ECA01BA717894FDB539A44D1D
:100520002F78CFCA920C1A99484C1196B54E412893
:10053000E4A6FE4B7291E7D4DD9F12E62938CE4542
:10054000AE02B824AEBDE9660862A22C2B00E223FD
:10055000D9C448E4D3ACBB34C7F0E34FB930EAA206
:1005600012F1302C36DE48F2B04C433F2E58E420D6
:10057000E358CD3122F0A22AE619905586F6557936
:10058000D1D7462FC0DC99E8F36ADF7FEB244A1EFF
:100590005A75DE2F5C19610353546A3B1870B64FCD
:1005A000F19C0A599D1992658C83142D448A75A972
:1005B000F590D2664EFA690F5B0B9865C8114259E7
:1005C0007FDD1B7517314C7558EB58637DF2A6C261
:1005D0006EB73F3E5E47ADB704E805F8B2CF19F3FA
:1005E000D285FE3E3EB162082C10070D739017FABB
:1005F0009B560275F951E0E91A7B9FB3F398B81C3A
:100600009CE1D535AEC860481109946BD08B15BC00
:100610000568D3548A51395C4276CED8AD8930C949
:10062000051CCC943F0F906F722D85649AB923F905
:100630000BC37C390F970797DA5848330523B882E4
:10064000E8D35389AF338022840C955C67B8770C6C
:100650005CA25F3D580F27F32FAE48BD0B6F54FBD4
:10066000674CEA3227F1FAE2B0EC0B15B470F65C95
:10067000DD7160C3C1A83265AC7A7741E5A96B1121
:1006800081FA348DFBC1806EC4603007D48B67BDA6
:10069000AA8C9C64ACDB0B248B636FE6BCE733A4B1
:1006A0004A4CA79F4353D2BB8F43C73D78683FA5B1
:1006B0003DCA6984A6972DC07D3134551D07B15FB1
:1006C000405C93B0BC7CB0BCE712EE6B2BD34D67A3
:1006D000703A9AF23C7C81FAD7D9909181B8B1F303
:1006E000486A264F0CCEB09EFD4A3AAFAC5B3FBF86
:1006F000445AA3191E4BE7366AD720AED77D3BE795
:10070000FF3A862ED04A3EAF9F8E01BFF84FC1E818
:100710006F74E145D3F7046A4B9DEC332776D7C558
:10072000E1B03B0E23ECF086D21ABF3D0462B36CFD
:10073000B2EB1705A60A8A7E831CB63709C60B7072
:100740003CB59381D893A05F1E08E2C6E5C972F15B
:10075000F1C1EDD5589383F865672E0DA9F16412A8
:10076000E64CEA153F8C1AB6BFF6B9523509B0E629
:10077000F7CDF1A5AA81D1816FB4A9661FFC48C04D
:10078000B6D18B062FF6EF1F0AE6CE3A4A55BF6D5B
:10079000F94DD408454BC366199210E1178E289184
:1007A00016BF3CEEA3A6999210E1F6CCACB8650B4F
:1007B0004366F8E3E53F2489475D7843D06117BD80
:1007C0005B645408455993F6958A4151624B510236
:1007D0003073C787C54BA2970FE8465F7E2AE1308A
:1007E00020B0FAE7CE6142576E21F37AECE325C7D9
:1007F00025F367A757400002CF1C807767BD70A123
:1008000019923175932727B682E4EB1D7848E7A546
:100810005E57EF6428641BF611B2039DB9180227D6
:10082000F7BE9D55FC00D2C7AEAD0BC5E9424148AD
:10083000D832CFF60FF5BC97C6994776BD89060F1B
:10084000630C51D45EEA48A8A2561C79848640887D
:10085000417655FCC2D7FDC9C7806135A74320F753
:10086000EB6C6613B0EC02753E4BAFB95D40DAD667
:100870006E2D3954C29535542572E178B8EBC11606
:10088000580F9C9BB4EA37EC3B11BAD58AA9E39880
:1008900000511C14E04096E5E9F22122B123607872
:1008A000D317F87AA5A8BA20D3151E32E45E1548EE
:1008B000AEA9E5B833ECE8A242ACBF108453871967
:1008C000B45F764D019D5674D95C97E788EA3ABFCC
:1008D000DC4C338A16B95BFAD842A7BB3C042778B4
:1008E00049812A5A7D7C23A8BAF79A9FD2663E385E
:1008F0003C75F9D13026306E5A6EDC6A693250335D
:10090000479EA4A86466F08AE4FD276F51258B43B7
:1009100074C98EBD8831BEEC65D2CB8D5A13481692
:100920008C610B11F6C666AEC3CC0CD2E19F82413E
:100930003F56F973EFDC3050CFB67FBCD0B310AB6D
:1009400024E4ECAD188C392D304CC5400DF6ACD6F6
:10095000185D96BF5F71759622970F02946EA6AED2
:100960006D8F1ECA129B2A1CCEA9EEFD128EFCEDC5
:100970000933BAF41A15F69D8716437C7857E1447B
:10098000C9EB1F584DC149115CB211A85516F1C6EB
:1009900050E98789F6CFD89C51A7BC5B316D4D518A
:1009A000D04CBC0D582D7B887AF98ED6404DBBBEFD
:1009B000C4E507FCD97B6DA642578F02944FE42A09
:1009C00065E2195A50E125654A60C2CDA8EC052EB2
:1009D000877B95B74FA00B1B4A7F92C890EE891E6C
:1009E00010D285E49F63C812BB4EB8CF0AEC184EF4
:1009F000E67CB33326C71FD20423EA070C5F90BD01
:100A0000A76A0F4AD610013C12292E96C04DBBBED4
:100A1000E5A783D56A3CE35BB8F25C6D1FA6F312D1
:100A200024F6D63B1014090782E8306A99DC950158
:100A30009CD4683BCA9812AB7725157D1032459837
:100A4000CD7ADF718A75C11CD46825EBBB54276F42
:100A50002AF7B9980327DE24A8BB98C284FF9B51CC
:100A6000D85350DAF588AA872FAED6EA6BDEC8D7FE
:100A7000A7286581E8B23B1D4F758F9F7A748EC1A0
:100A80005F9AA89DFA03A3719B376DD50BF5E1A181
:100A90001B016AC667AAEA2C9DA4D26EFCDE2E7FDB
:100AA0009469E54AE001483C6BF71EB60B5FF92EEE
:100AB00007C5E8AE371BBC3CD8D50B919E8024F50A
:100AC000060C0E9807962D19DC5893CCFB4EEBBD07
:100AD0000FF5AF01FAF17C438CB8563EBE774E2B32
:100AE000F7BBB74547CDCCA64C727B6A2A7013077B
:100AF000FDB89C983AD823675B34D5140CAB771FAC
:100B0000F83D5A9F92B72CAD31DE6107B36BF738D1
:100B1000159546144853695266076D83718A672597
:100B2000200FFED702D76E2CD21A0A5DFD0F74E398
:100B3000A436079ADFD479BFEF59C04452879A6E22
:100B40001D0EEEDE2E1AA98F3AC9BAEC99782D55F2
:100B50006B14C206D5FC93534D118CF8FA797CA620
:100B600064AE61B87B9456A639789AE5C7DF1863FE
:100B7000239CFA66BBB75A274CD1A18322B35249B2
:100B800035B022835912001698DDADC294F9D37B9B
:100B9000647F443E3C8B9A839C696BE4DF9FED54F9
:100BA0001FE55D7A0582B3DDEFFC5396B02C5AF851
:100BB000DF9C8B164EDFDA4D090969500365D87347
:100BC00070E886BFBB35CEB246CB02005BB4E2C64E
:100BD0008F2F98AF874B4845EDCC1DE658D6F25085
:100BE000259F52C7CB8A179D5BE5C8D772B752B213
:100BF000C498E37A173EC660A797B0CF1881538494
:100C00004CD51732031339510910E377494F62016C
:100C1000BF8C9AE0419E897436F996862E961C4ABE
:100C2000B72B4A97BC9940A3E03DC8AD2FDF4F2CAE
:100C3000C469829F9B810C615CA59D8C89C02CB48A
:100C40004A334EEBA25640C0C246AF6AFC67D18021
:100C50005EC56D8443273F5515966AA0A5DAB7FF98
:100C6000B7756E4C49919D22A346EAED9A00E23297
:100C7000C3D6A9712055A319EDF84FA7129C66871A
:100C8000AF4EB7F0DBBFEFF0F6AFEADA09FEDE38C1
:100C90005CA5A2DF9945A8E4E792AC67AA4FBF77AD
:100CA0003EA24049224A1E3BAA707F95AF374BFCBB
:100CB00099E2E0BAD734CE55885B841B57C48003D1
:100CC00053C92F93044DD596E570A66E635D9D6C58
:100CD000DB020AA9DA8B53DCD99AC5942C91922AAB
:100CE000DEBB8B13B9199664CCF26439B77549E948
:100CF00086C28662D924D3813549FCA0A5A093057C
:100D000064B41A57CE0C900227C57A2B5DAE3ED53F
:100D1000DD107C14EA3A08AC724E903D3B7C862E86
:100D2000EBD40670E6C7FB5FBD18F411A41A93C399
:100D3000BED9FB26482F373CD003471AF762192447
:100D40005CF4A892207AF29E2AC595A2FBA4EA85BB
:100D5000D856B770D16030A5308270DC7A658A369B
:100D60003F5B0CAE547CD357847B3A651881EE050B
:100D70009B444DB8DAA2A1C915D373030E43E98E83
:100D800015F9BEC6C58AE5C01EC2379E2A26A5A093
:100D9000BD245FB9C1AB3448B95D98B46518F3633D
:100DA00019441B1116FFDCF17908860F529873C4A1
:100DB00092902B4709D0436C2F20EBDCDAC5087BDF
:100DC0009442306AC7DA8CC376A7A5CC6213006060
:100DD0003158449BF56414F511C5545283D4730102
:100DE000160EB37A29693556D4EE8A17A299249C37
:100DF000D78FDB55B53E10034F00640064006200DE
:100E000061006C006C000000220341006C00650072
:100E1000780061006E0064006500720020005400DC
:100E200075006C006C006F0068000000040309048A
:100E300009023B00020100A0FA09040000010301BD
:100E4000010009211101000122400007058103086A
:100E50000001090401000103000000092111010043
:100E600001227B000705820320000112010002001D
:100E7000000008EDFE49CA01000102000105010958
:100E800002A10185020901A100050919012908151E
:100E90000025019508750181020501093009311508
:100EA00081257F95027508810609381581257F9572
:100EB0000175088106050C0A38021581257F950108
:100EC00075088106C0C005010980A10185031901CB
:100ED0002AB700150126B700950175108100C005DD
:100EE0000C0901A101850419012AA002150126A0FF
:100EF00002950175108100C005010906A1010507D1
:100F000019E029E715002501950875018102950171
:100F1000750881010507190029FF150026FF0095B6
:100F200006750881000508190129059505750191C7
:100F300002950175039101C011241FBECFEFDAE0C5
:100F4000DEBFCDBF11E0A0E0B1E0EEECFAE502C0FB
:100F500005900D92AA3AB107D9F722E0AAEAB1E0CA
:100F600001C01D92AA3AB207E1F70E94531C0C94EB
:100F7000652D0C940000CF93DF93662359F0EC01AC
:100F80000E94881D60E070E0CB01BE01DF91CF912F
:100F90000C943814DF91CF910895EF92FF921F9334
:100FA000CF93DF9300D000D000D0CDB7DEB7182F9D
:100FB0007B010E94481D29834B835C836D837E8364
:100FC000F7018081882319F0512F532B03C010950E
:100FD000512F532349816B817C818D819E810E9499
:100FE000691D26960FB6F894DEBF0FBECDBFDF9108
:100FF000CF911F91FF90EF900895CF92DF92EF92E3
:10100000FF920E94B0198823A9F00E9434146B014A
:101010007C01672B41F480EAC82E8FE0D82EC701EF
:10102000B6010E943814C601FF90EF90DF90CF9078
:101030000C94881DFF90EF90DF90CF900895EF9271
:10104000FF920F931F93CF93DF93CDB7DEB72C970B
:101050000FB6F894DEBF0FBECDBF4F835887162F53
:101060006987072F7A878B879C877C010E94B0193C
:10107000882369F18091AE01882301F18091AD014F
:10108000810F8093AD019091AC01090F0093AC01E9
:101090003CE0632F0E94D32C282F802F632F0E94C7
:1010A000D32C222321F0F22EF1941092AD0188234B
:1010B00041F0E82EE1941092AC0103C0612F6195DC
:1010C00002C000E060E069870A87EB86FC8686E064
:1010D000FE013796DE01119601900D928A95E1F797
:1010E00029813A814B815C816D817E8180E090E035
:1010F0002C960FB6F894DEBF0FBECDBFDF91CF9117
:101100001F910F91FF90EF9008950F931F93CF932E
:10111000DF938C01EB010E94E508882309F44EC09F
:10112000053F1105E1F1C0F4023F110561F148F4FA
:10113000013F110509F042C0BE016E5F7F4F81E0A3
:1011400026C0033F110531F1043F1105B9F5BE0179
:101150006E5F7F4F88E01BC0083A9DE5190721F1BB
:1011600038F4073A1D4551F58A818093AE0125C0B8
:10117000093A9DE51907E1F00A3A1D45F9F46A813B
:1011800080E49FE118C0BE016E5F7F4F82E00E9445
:10119000CD0713C0BE016E5F7F4F84E0F8CFBE0164
:1011A0006E5F7F4F80E1F3CF6A8180ED97E003C0EF
:1011B0006A8180EA9FE00E94BB0780E0DF91CF91C7
:1011C0001F910F91089581E0089581E00895089599
:1011D0000C94E7081F93CF93DF9300D000D01F92A9
:1011E000CDB7DEB749835A836B833091B0018981D3
:1011F0009A81311114C0662359F0222349F00E94CC
:101200007A0F182F682F89819A810E94210F03C0BD
:101210000E944D0F182F69817A81812F04C00E948E
:101220007A0F69817A810F900F900F900F900F9035
:10123000DF91CF911F910C949316FC01262F4081D2
:1012400051816281738184810C94EA0881E0089560
:10125000CF93DF93EC0160E00E941D09BE01DF9196
:10126000CF910C94E8080C9400180C94FC17089586
:101270000E94CB0D0E9437092FEF84E39CE02150A0
:1012800080409040E1F700C000000C94CA250F9305
:101290001F93CF93DF938C0161E00E941D09EC0145
:1012A000B8010E9485088823F1F1B801CE010E949F
:1012B000BC208823C1F1B801CE010E94D01E882332
:1012C00091F1B801CE010E941820882361F1F80144
:1012D0008281882309F1CB358DE5D807C1F050F420
:1012E000C115FCE5DF0781F0CF3DDC45A9F40E9484
:1012F000AF1419C0CC35EDE5DE0761F0CD35DD4525
:1013000059F40E94F41308C00E9438090CC00E94CE
:10131000FD1302C00E940014C801DF91CF911F91FC
:101320000F910C94E30880E0DF91CF911F910F9112
:1013300008950E94E3240E94B4090C94D91C0E94D1
:10134000B7090C94E92408950C94A30981E0089549
:101350000C94A6090895CF93C82F0E94A4098C2F3E
:101360000E94A809CF91089580E00C94AB090E94D7
:1013700021240C94AB090E9421249091AF0189177C
:1013800021F08093AF010C94AB090895CF93DF93C4
:10139000CDB7DEB72B970FB6F894DEBF0FBECDBF2B
:1013A0004F83588769877A878B8761110E94401322
:1013B0009E012F5F3F4F86E0F90111928A95E9F770
:1013C00085E0FE013796D90101900D928A95E1F7EB
:1013D00089819A814C815D81452B31F09F3F31F4A9
:1013E00091E08F3F19F403C091E001C090E090FFBD
:1013F00009C049815A816B817C818D819E810E94C7
:10140000611205C0C9010E9426098111F2CF2B96F5
:101410000FB6F894DEBF0FBECDBFDF91CF91089518
:10142000FC01808191810E94BC0F0895CF93882395
:1014300009F49CC0C82F8238C1F40E94212481FD88
:1014400095C069E380910201909103010E94BB2441
:101450000E9462132FEF81EE94E021508040904073
:10146000E1F700C0000069E319C0833801F50E946C
:10147000212480FD7BC063E58091020190910301EE
:101480000E94BB240E9462132FEF81EE94E0215052
:1014900080409040E1F700C0000063E580910201C8
:1014A000909103010E94BD24CF910C946213843863
:1014B000C1F40E94212482FD59C067E48091020199
:1014C000909103010E94BB240E9462132FEF81EED2
:1014D00094E0215080409040E1F700C0000067E4B4
:1014E000DDCF8CEF8C0F813AD0F46C2F809102010C
:1014F000909103010E948524882349F06C2F8091EC
:101500000201909103010E94BD240E9462136C2F7E
:1015100080910201909103010E94BB24C5CF80E21B
:101520008C0F883048F4C77081E001C0880FCA95DD
:10153000EAF70E942313B8CFEBE5EC0FE33040F459
:10154000F0E0EF59FE4F808190E0CF910C944D2454
:10155000C85AC73158F4EC2FF0E0EE0FFF1FED5CD6
:10156000FE4F80819181CF910C946324CF91089597
:10157000882309F45BC0682F823879F40E94212403
:1015800081FF54C069E380910201909103010E94A0
:10159000BB240E94621369E310C08338B1F40E9437
:1015A000212480FF43C063E58091020190910301F3
:1015B0000E94BB240E94621363E580910201909116
:1015C00003010E94BD240C946213843879F40E94B4
:1015D000212482FF2BC067E48091020190910301D6
:1015E0000E94BB240E94621367E4E7CF8CEF860F52
:1015F000813A18F380E2860F883048F4677081E002
:1016000001C0880F6A95EAF70E942913DCCF8BE5A9
:10161000860F833020F480E090E00C944D24685ACB
:10162000673120F480E090E00C94632408951F93C8
:10163000CF93DF93182FEB010E94160A209741F0F9
:101640008FE99FE00197F1F700C000002197F6CFE6
:10165000812FDF91CF911F910C94B80A893319F033
:1016600060E070E002C060E570E00C94170B882326
:1016700021F00E9423130C9462130895882321F013
:101680000E9429130C9462130895CF92DF92EF9277
:10169000FF920F931F93CF93DF937C01D62FC72F19
:1016A000FC011281058102950F700E941913882395
:1016B000B9F01123A9F08C2F807F803421F080E2D3
:1016C0008D0F883068F080917C0282FD09C082E035
:1016D0000E94C2130E94191391E0D82ED92601C08E
:1016E000D12CCC2EC2948FE0C8228C2D90E08C306F
:1016F000910508F0C4C1FC01EA5AFF4F0C94F52C87
:101700008C2F807FCF70882311F0C295C07F11236A
:1017100099F0CC2309F49FC180E28D0F883010F03E
:10172000D11104C08C2F0E94231303C08C2F0E9460
:1017300033130E9462138FC18D2F0E94B80ACC23ED
:1017400009F49DC180E28D0F883038F1DD2329F145
:101750008C2F0E94391324C08C2F807FCF70803251
:1017600011F0C295C07FDD2319F0D130A1F13DC049
:1017700080917C0282FF17C0112349F0CC2329F00D
:101780008C2F0E9423130E94621380E065C180E0C9
:101790000E94B80ACC2309F472C18C2F0E9429132D
:1017A0000E9462136CC1112371F0002341F00130DB
:1017B00031F40E9443138C2B0E944B1360C10E9492
:1017C00043138C2B1DC0002319F0013009F457C1BD
:1017D0000E94581325C0112321F0063008F04FC194
:1017E0000EC0053008F04BC11BC0112361F000236F
:1017F00031F0F701858180FF2EC18F7085838C2F9A
:101800000E94370B3CC1002359F0D93309F034C191
:10181000FFEF07EE13E0F15000401040E1F72AC15E
:101820008C2F0E943E0B2BC18C2F86958695837042
:1018300019F0813061F023C1112321F08D2F9C2FED
:10184000937002C080E090E00E944D2420C11123DB
:1018500021F08D2F9C2F937002C080E090E00E94B9
:10186000632415C18C2F837009F047C011110BC17F
:101870002D2F229526952770220F220F6D2F6F7026
:10188000862F90E0A0E0B0E0022E04C0880F991FE0
:10189000AA1FBB1F0A94D2F7D4FF10C04FE050E03C
:1018A00060E070E004C0440F551F661F771F2A9543
:1018B000D2F7409550956095709503C040E050E098
:1018C000BA01C695C695C3708A019B01082B192BD6
:1018D0002A2B3B2BC901B801C23049F058F4C13062
:1018E00019F00E94370ECFC00E94250ECCC00E9476
:1018F000490EC9C00E94230EC6C0112319F08C2FB7
:10190000817001C08695882309F4BDC02D2F2295D2
:1019100026952770220F220F6D2F6F70862F90E073
:10192000A0E0B0E0022E04C0880F991FAA1FBB1FC1
:101930000A94D2F7D4FF10C04FE050E060E070E0AE
:1019400004C0440F551F661F771F2A95D2F7409594
:1019500050956095709503C040E050E0BA01C6957F
:10196000C695C3708A019B01082B192B2A2B3B2B90
:10197000C901B801C23049F058F4C13019F00E94D1
:10198000FC0E81C00E94EA0E7EC00E940E0F7BC03A
:101990000E945D0E78C0CF70112339F08C2F0E9409
:1019A000830E8D2F0E94370B6EC08D2F0E943E0B31
:1019B0008C2F0E94A40E67C0D23F21F128F4D03FA3
:1019C00041F0D13FC1F043C0D33F19F1D43F79F08A
:1019D0003EC0112341F0053008F051C08C2F8F71AB
:1019E0000E94C90E4CC0063008F049C0F7CF809164
:1019F0007C0282FF18C0112339F08C2F8F710E9456
:101A0000830E3DC01123C9F38C2F8F710E94A40E49
:101A100036C0112329F08C2F8F710E946E0E2FC0BB
:101A20000E94690E2CC0112349F0CF718C2F0E94A7
:101A3000830E63E08C2F0E94A71321C081E00E94D7
:101A4000C2130230E0F082E00E94C21318C01123DA
:101A500031F0002391F28D2F0E94160A10C000234E
:101A600099F2D93349F41FEF27EE33E011502040AB
:101A70003040E1F700C000008D2F0E94B80A88EFC7
:101A80008C0D843020F40E9421240E94AB09DD20BB
:101A9000C9F00E94151380FD15C0F70112820E9443
:101AA0000F130E94830EC7010E94830D0E940F1323
:101AB000DF91CF911F910F91FF90EF90DF90CF902A
:101AC0000C94A40EDF91CF911F910F91FF90EF9096
:101AD000DF90CF9008950F931F93CF93DF93EC0186
:101AE000688179818A810E94C70F8C010E94200F32
:101AF0000E94110EB801CE010E94450BDF91CF91DB
:101B00001F910F910895CF93DF93EC019881898104
:101B10002B813C81232B31F08F3F31F481E09F3FBB
:101B200019F403C081E001C080E080FD1DC0CE013A
:101B30000E944709811110C00E9419138823A1F047
:101B40008A81882389F080917C0282FD0DC082E029
:101B5000DF91CF910C94C213CE010E946B0DCE0188
:101B6000DF91CF910C942809DF91CF91089580E007
:101B700090E00E944D2480E090E00E9463240E9447
:101B800040130C94621380910201909103010E9412
:101B9000BF240C94B70D0E9430130C94C30D929582
:101BA0009F70963079F010F4925001C09A509230A4
:101BB00068F4803F69F018F4883E40F409C0843F1F
:101BC00029F406C0883E20F0813F11F080E008959E
:101BD00081E00895FC01808191810E94BC0F0E94E8
:101BE000CF0D0895CF93DF9300D000D01F92CDB7D3
:101BF000DEB70F900F900F900F900F90DF91CF9165
:101C00000895CF93DF9300D000D000D0CDB7DEB7DA
:101C100026960FB6F894DEBF0FBECDBFDF91CF91F1
:101C20000895089508950C94120E0C94130E0E94BA
:101C3000150E6093D3017093D4018093D5019093D6
:101C4000D6010C94B70D0C94170E0F931F930091AF
:101C5000D3011091D4012091D5013091D601602B90
:101C6000712B822B932B1F910F910C94170E0F93B6
:101C70001F930091D3011091D4012091D50130918F
:101C8000D60160237123822393231F910F910C941B
:101C9000170E0F931F930091D3011091D40120913F
:101CA000D5013091D60160277127822793271F9194
:101CB0000F910C94170E0C94120E0E945B0E609301
:101CC000CF017093D0018093D1019093D2010C94F5
:101CD000B70D60E070E0CB010C945D0E0F931F9385
:101CE00041E050E060E070E08A019B0104C0000F19
:101CF000111F221F331F8A95D2F7C901B8011F9106
:101D00000F910C945D0E0F931F9341E050E060E043
:101D100070E004C0440F551F661F771F8A95D2F7E5
:101D20008091CF019091D001A091D101B091D201C9
:101D30008A019B01082B192B2A2B3B2BC901B801C7
:101D40001F910F910C945D0E0F931F9341E050E093
:101D500060E070E004C0440F551F661F771F8A952E
:101D6000D2F740955095609570958091CF019091F4
:101D7000D001A091D101B091D2018A019B01082329
:101D800019232A233B23C901B8011F910F910C94F9
:101D90005D0E0F931F9341E050E060E070E004C0DF
:101DA000440F551F661F771F8A95D2F78091CF0188
:101DB0009091D001A091D101B091D2018A019B01F3
:101DC000082719272A273B27C901B8011F910F911E
:101DD0000C945D0E0F931F930091CF011091D001D1
:101DE0002091D1013091D201602B712B822B932B4A
:101DF0001F910F910C945D0E0F931F930091CF01D3
:101E00001091D0012091D1013091D2016023712332
:101E1000822393231F910F910C945D0E0F931F93B8
:101E20000091CF011091D0012091D1013091D201C8
:101E300060277127822793271F910F910C945D0EC5
:101E40000895292F220F920F990F890FE82FE695F9
:101E5000E695E695877051E001C0550F8A95EAF73F
:101E600085E0E89FF0011124EF54FE4F20E030E0C0
:101E700070E04081CB01022E02C0969587950A94AE
:101E8000E2F78170819584278523842781932F5FD2
:101E90003F4F2530310569F70895292F220F920F02
:101EA000990F890F682F669566956695982F97709C
:101EB00085E0689FB001112440E050E080E0FB0124
:101EC000E40FF51FEF54FE4F208130E0092E02C0D1
:101ED000369527950A94E2F721703327042E01C026
:101EE000220F0A94EAF7822B4F5F5F4F453051056E
:101EF00031F70895BF92CF92DF92EF92FF920F9346
:101F00001F93CF93DF938C01C090CF01D090D0016D
:101F1000E090D101F090D2018091D3019091D40151
:101F2000A091D501B091D601C82AD92AEA2AFB2A64
:101F3000CFE1D0E0D701C6010C2E04C0B695A7951D
:101F4000979587950A94D2F780FD04C0219790F762
:101F5000B12C07C0BC2EB8018C2F0E94A616019789
:101F6000A9F38B2DDF91CF911F910F91FF90EF90EF
:101F7000DF90CF90BF900895CF93DF93EC010E9444
:101F80007A0FBE010E94A616DF91CF9108951F938C
:101F9000CF93DF93EB019091B001992321F0CB0116
:101FA0000E94BC0F13C0882349F0CB010E947A0F16
:101FB000182F682FCE010E94210F04C0CB010E9470
:101FC0004D0F182FBE01812F0E94A616DF91CF91D1
:101FD0001F9108951F93CF93DF93C091D70116E00F
:101FE0008091D801C81799F0D0E01C9FF0011D9F87
:101FF000F00D1124E752FE4F4081518162817381BF
:10200000848195810E94010E2196C770E9CFDF91EE
:10201000CF911F9108954091090250910A02609159
:102020000B0270910C0280910D0290910E020C94A3
:10203000010EEF92FF920F931F93CF93DF93809146
:102040000E0282958F7009F065C080910B02882383
:1020500009F460C08091D701F090D8011091090275
:1020600000910A0260910C0270910D0291E01F3FF5
:1020700009F090E0C0910001D0910101292F96E074
:10208000E92E8F1509F446C06115710521F00F3F47
:1020900021F030E003C031E001C0322F90E030FD8C
:1020A00036C0E89EF001E99EF00D1124DF01A75231
:1020B000BE4F11963C911197301329C03C913113BA
:1020C00026C012963C911297311121C013964D9162
:1020D0005C911497461B570B4C175D07C0F4809119
:1020E0000E028F70806180930E02E252FE4F80815B
:1020F0008F708061808389E092E00E94830DDF9180
:10210000CF911F910F91FF90EF900C94EA0F0196E1
:102110008770B7CFDF91CF911F910F91FF90EF9014
:1021200008959F92AF92BF92CF92DF92EF92FF926B
:102130000F931F93CF93DF93CDB7DEB761970FB6A1
:10214000F894DEBF0FBECDBF8C0185E0F801DE0143
:102150001D9601900D928A95E1F7D8011296EC90A8
:1021600090910902E0910A0220910C0230910D0237
:102170002115310531F0EF3F31F481E09F3F19F433
:1021800003C081E001C080E0B82FB1709B2E80FDBC
:1021900047C1D8014C9111965C9111971396AD905F
:1021A000BC90149789E0C82E82E0D82EF0900B02E4
:1021B000B501621B730B2091000130910101FF20DA
:1021C00009F4D9C080910E026217730708F095C018
:1021D000282F207F09F052C05E1313C0491311C08D
:1021E000FE2CE1100EC08F70806180930E020E9461
:1021F0000B10C6010E94830D80910E02F8018583A9
:102200004DC1AB2831F05F3F31F481E04F3F19F40D
:1022100003C081E001C080E080FD03C081E08E2525
:1022200002C080E090E0F82FF170FF2E80FF1CC00C
:102230008091D7012091D80136E0821709F40BC1B3
:1022400090E0389FF001399FF00D1124E752FE4FC6
:102250006181561306C06081461303C06281E61295
:1022600003C001968770E9CFFE2CEE2009F416C159
:1022700080910E02816080930E0254C05E1306C0EE
:10228000491304C0E11002C0F80199C0C8010E94BE
:10229000EA0D882361F1EE2051F120910E02822F88
:1022A00082958F7090E0029774F08091090290916E
:1022B0000A0298878F831986BB86AA862C87CE014F
:1022C00007960E94830D86E0F801A9E0B2E0019034
:1022D0000D928A95E1F70E9419100E940B100AC016
:1022E0005E1711F1C8010E94EA0D81112CC0C801CE
:1022F0000E94830DFF24F394D1C0282F207F81F703
:102300007A2DB98AA88A6E2D89890E94F20D89E0FA
:1023100092E00E94830D86E0D6011D928A95E9F72E
:102320000E940B10F12CBAC04913DCCFE110DACFB8
:10233000F8018583C8010E94830D86E0D6011D92B5
:102340008A95E9F7ABC0EE2091F220910E02822F20
:1023500082958F7090E002970CF4B5CF80910902BE
:1023600090910A029A8389831B82BD82AC822E835C
:10237000CE010196A6CF6217730708F044C0FE2C69
:10238000EE2009F4B4CF5E1330C049132EC0209163
:102390000E0220FD21C0822F82958F70482F50E0C1
:1023A00041155105C9F0F80125834F30510541F021
:1023B0008F5F982F9295907F822F8F70892B8583C6
:1023C000C8010E94830D86E0F801A9E0B2E0019007
:1023D0000D928A95E1F73CC086E0F801A9E0B2E0F1
:1023E00001900D928A95E1F759C0C8010E94EA0D4B
:1023F000811169CF80910E02816080930E02C80125
:102400000E94830D4BC07A2DB98AA88A6E2D8989C6
:102410000E94F20D86E0D6011D928A95E9F718C058
:10242000EE2009F464CFC8010E94EA0DF82E88233B
:1024300009F45DCF86E0F801A9E0B2E001900D92C9
:102440008A95E1F789E092E00E94100A0E94191033
:102450000E940B1023C04D875E878D859E850E944C
:10246000BC0F292F22952F70223028F49F7039F04D
:10247000811105C00BC0243028F49F7049F4805EA0
:10248000883020F0C8010E94830D9F2CF92C06C0D3
:10249000D80115969C91907F91F7F8CF8F2D61967A
:1024A0000FB6F894DEBF0FBECDBFDF91CF911F9165
:1024B0000F91FF90EF90DF90CF90BF90AF909F90E3
:1024C00008951F93CF93DF93CDB7DEB72C970FB648
:1024D000F894DEBF0FBECDBF4F83588769877A87D8
:1024E0008B879C87CE0107960E9491108823D1F09C
:1024F0009F8188852A853B85232B31F08F3F31F4DE
:1025000081E09F3F19F403C081E001C080E080FDBD
:1025100047C04F81588569857A858B859C850E9447
:10252000010E3EC086E0FE013796DE011196019055
:102530000D928A95E1F7FF81E8856A857B856115B3
:10254000710531F0EF3F31F481E0FF3F19F403C032
:1025500081E001C080E080FD23C02091D80130E0FF
:10256000C9010196877099274091D70150E08417DF
:102570009507F1F1F983EA837D836C8396E0929F5E
:10258000D001939FB00D1124A752BE4FFE0131968A
:1025900001900D929A95E1F78093D8010E94EA0F7D
:1025A00016E08091D7019091D801891771F1189F99
:1025B000C001112487529E4F0E949110882329F157
:1025C000E091D7011E9FF0011124E752FE4F408198
:1025D000518162817381848195810E94010E809175
:1025E000D70190E00196877099278093D701D9CFC2
:1025F0000E94CB0D1092D8011092D701E9E0F2E0D1
:1026000086E0DF011D928A95E9F72C960FB6F894C3
:10261000DEBF0FBECDBFDF91CF911F910895809196
:102620001702859585958595089580911702877085
:10263000089590911702977081E009F480E0089561
:1026400080912202089590912202892B8093220288
:102650000895809590912202892380932202089503
:1026600010922202089590912102892B80932102D9
:1026700008958095909121028923809321020895E5
:1026800010922102089580911802089508950C94E3
:1026900046130C94471390917C0292FD08C09091D0
:1026A0001802981721F0809318020C94491308958A
:1026B00080911802882329F01092180280E00C946F
:1026C00049130895CF93DF93E0910201F091030144
:1026D000809122028083E0910201F09103019081B8
:1026E00080912102892B808380911802882381F0B8
:1026F000E0910201F09103019081892B8083809108
:102700000201909103010E94792481110E945813C3
:10271000C0910201D091030148E050E06FE072E007
:10272000CE010E94072D892B69F088E0FE01AFE001
:10273000B2E001900D928A95E1F7CE01DF91CF9141
:102740000C943424DF91CF9108950C94461390910A
:102750007C0292FD10C098E0899F90011124262BE5
:10276000209317020E94830E80911702859585950C
:1027700085950C94A5130C94830E1092170280E09B
:102780000C94A51320911702809582238093170241
:10279000982F977099F430E0482F082E000C550BB5
:1027A0002417350759F090917C0292FD07C085955A
:1027B000859585950E94A40E0C94BD130895909163
:1027C0007C0292FB222720F9281769F080FB92F9FE
:1027D00090937C0280917B0290917C020E9427144E
:1027E00082E00C94C213089580917C0282FB8827BA
:1027F00080F991E089270C94DF1381E00C94DF13BA
:1028000080E00C94DF1380E090E00E942B2D21E00B
:10281000893E9E4F09F020E0822F089582E090E0EB
:102820000C941D2D83E090E00C941D2DCF9384E03B
:1028300090E00E941D2DC82F82E290E00E941D2D85
:102840002C2F30E0A901582BCA01CF910895CF93C6
:10285000C92F682F84E090E00E94312D6C2F82E216
:1028600090E0CF910C94312D8FE090E00C94252DC9
:10287000AB01BC018FE090E00C94432DAB01BC0197
:1028800083E190E00C94432D60E070E0CB010C9468
:102890003E1460E070E0CB010E9438140C944414A4
:1028A00069EE7EEF80E090E00E944F2D60E082E0D4
:1028B00090E00E94312D60E083E090E00E94312D95
:1028C0001092D3011092D4011092D5011092D6012A
:1028D00060E084E090E00E94312D60E082E290E0D0
:1028E0000E94312D60E085E090E00E94312D60E093
:1028F00086E090E00E94312D6FEF87E090E00E942B
:10290000312D40E050E0BA0188E090E00E94432D74
:1029100060E08DE090E00E94312D40E050E0BA018F
:1029200088E190E00E94432D60E087E190E00E9402
:10293000312D40E050E0BA018CE190E00E94432D3F
:1029400060E070E080E290E00E944F2D40E050E0B7
:10295000BA0188E190E00E94432D0C9449140C9434
:102960005014682F8EE090E00C94312D0E946D255C
:1029700060932F0270933002809331029093320261
:1029800060932B0270932C0280932D0290932E0261
:10299000089585B7806885BF85B7806885BF08952D
:1029A0000C94B01908950C94D2140C94D2140C9475
:1029B000D5140C94D2140C94D9140C94D2140E94F3
:1029C000C91483EC97E10E9417240E94DD140C9433
:1029D000DB140E94D3140C94D2140E94C6170C94DA
:1029E000AA090E9458250E9482170E94D8190E94A5
:1029F00001190E94ED140E94B81E0E94961C0E94AC
:102A0000E2190C94D7148F929F92AF92BF92CF92FB
:102A1000DF92EF92FF920F931F93CF93DF93CDB787
:102A2000DEB72A970FB6F894DEBF0FBECDBF0E9467
:102A30002519982E81110E94B61483E2A82E82E0F7
:102A4000B82E00E010E0802E802F0E94EA17D82ECA
:102A5000F501C1905F01C826B1F40F5F1F4F083028
:102A6000110589F78FEF89838A831B820E94612574
:102A70008160782F9D838C8349815A816B818D8100
:102A80000E94C6092FC08091330281FD0E94F01779
:102A9000E12CFF24F3948C2D8F21F1F00E94D014AF
:102AA000882399F0EE828F82DF2081E009F480E0B4
:102AB00088870E9461258160782F9A8789874E8157
:102AC0005F8168858A850E94C609F801ED5DFD4F2A
:102AD0008081F826F08206C0E394FF0CF6E0EF1246
:102AE000DACFBBCF81E0911001C080E02A960FB60B
:102AF000F894DEBF0FBECDBFDF91CF911F910F9134
:102B0000FF90EF90DF90CF90BF90AF909F908F900D
:102B100008950E9403150E94B0190E94D91C0C94BC
:102B2000BB09CF93DF930E94AB16EC01811522E520
:102B30009207E8F5811531E5930708F0B6C0883EA5
:102B4000910528F5803E910508F0E9C0883A910585
:102B500070F4853A910508F07AC08130910509F446
:102B600073C008F4D9C0049708F0D9C0D5C08F3B12
:102B7000910508F0D1C0C85AD0E0CC0FDD1FCC5968
:102B8000DE4F0990D881C02DCE019464C9C0811553
:102B900040E5940708F069C0811550E4950708F0F6
:102BA00060C09A9581159F4108F4B9C0B5C08115E0
:102BB00036E5930728F5811545E5940708F092C09E
:102BC000811554E5950708F087C0AC01437055277F
:102BD000282F26952695C115D34508F06CC081E0B5
:102BE00090E002C0880F991F4A95E2F740E2249FC7
:102BF00090011124EC01C22BD32BCE019C6890C014
:102C000081152AE5920780F4811539E5930708F0CC
:102C100072C0811548E5940708F47EC0D82FCC27F0
:102C2000CE01806F906A7CC090568115904208F06A
:102C300073C08D2F8F710E943F17DD27D0628F7177
:102C4000AE01582BCA016CC081E090E069C0C55A42
:102C5000D0E0CE56DE4F8881C82FD0E0CE01906400
:102C60005FC0DF70CE01906A5BC074E09695879577
:102C70007A95E1F7282F23703C2F337081E090E0A4
:102C800002C0880F991F3A95E2F79C68AC01522B5D
:102C90009A019C2F9F709695969550E2959FE00122
:102CA0001124C9018C2B9D2B3BC0D82FCC27CE01E2
:102CB000816F906A35C081E090E002C0880F991F53
:102CC0004A95E2F750E2259F90011124EC01C22BB6
:102CD000D32BCE019A6824C0D82FCC27CE01846F85
:102CE000906A1EC00E943F178F7190E0D82FCC27AA
:102CF000CE01906215C08F700E943F1794E0D69568
:102D0000C7959A95E1F7CF70D0E0DC2FCC27D0693A
:102D10009E01282BC90104C080E090E001C0CE01D3
:102D2000DF91CF91089520E3829FC0011124FC011F
:102D300026E0729FE00DF11D1124E60FF11DEE0F4C
:102D4000FF1FE852FF4F8591949108950E949316BA
:102D50000E94911508958238910569F1B0F481338C
:102D6000910509F46DC048F48932910509F463C0F6
:102D70008A32910509F469C008958533910509F4F3
:102D800055C089339105B9F00895833E910569F1E5
:102D900038F4803E9105B1F0823E910509F1089525
:102DA000863E9105A9F1873E9105B9F1843E9105D2
:102DB00009F064C023C020917B0220FD4FC021FD9B
:102DC0004DC0089580917B0280FD44C080917C02BB
:102DD00080FF44C080917B0284FD42C083EE4DC0E1
:102DE00080917B0282FF38C0F5CF80917B0282FD0B
:102DF00033C080917C0280FD31C0ECCF80917C0299
:102E000081FF32C080917B0284FD2AC087EE35C0ED
:102E100080917B0283FF26C0F5CF80917B0283FDEA
:102E200021C080917C0281FD1FC0ECCF80917B028C
:102E300085FD1CC01DC080917B0285FD19C016C098
:102E400080917B0286FD16C017C080917B0286FDB3
:102E500013C010C089E311C082EE0FC080EE0DC018
:102E600080E00BC086EE09C084EE07C089E205C091
:102E700085E303C08AE201C081E390E00895909168
:102E80007B0292FF0DC0282F2871283019F4877F0C
:102E9000846006C0282F2471243011F48B7F886051
:102EA00093FF0DC0282F2871283119F4877E846183
:102EB00006C0282F2471243111F48B7E8861209163
:102EC0007C0220FF0DC0382F3871383019F4877F0D
:102ED000816006C0382F3171313011F48E7F8860E7
:102EE00021FF0DC0282F2871283119F4877E8161B8
:102EF00006C0282F2171213111F48E7E886194FD46
:102F0000877E0895109277021092780210927902CB
:102F100010927A020895CF92DF92EF92FF926B01A6
:102F20007C010E94B01981110EC00E946D25C61A45
:102F3000D70AE80AF90AC0927702D0927802E092A2
:102F40007902F0927A02FF90EF90DF90CF9008958F
:102F50000F931F930E94B019882321F01F910F91A6
:102F60000C946D250E946D250091770210917802D6
:102F70002091790230917A02600F711F821F931F96
:102F80001F910F91089580E0089508950E94031401
:102F9000811102C00E94AF140E940E14809333026C
:102FA0000E94161490937C0280937B020E94C517A6
:102FB0000E941214682F70E080E090E00E94230EBF
:102FC0006091CF017091D0018091D1019091D20197
:102FD0000C945B0EE82FF0E0EA57FD4F80810895D6
:102FE000089580EA8A95F1F7089500C008950C9439
:102FF000F11708950C94F9170C94FA170C94F9171B
:103000000C94FE170C94F9170F931F93CF93DF9333
:1030100000D000D0CDB7DEB70E94B01960918E020B
:103020008823E9F119821A821B821C82862F90E084
:103030008E010F5F1F4FB8018A579D4F0E94F019F4
:10304000882389F080917D0290E044E050E0B8014F
:103050008A579D4F0E94072D21E020933402892B2F
:1030600069F410E019C0809134028823D1F384E020
:10307000F80111928A95E9F710923402E0917D02ED
:10308000F0E0EA57FD4F89819A81AB81BC81808352
:103090009183A283B38311E00E9435090DC070E0D3
:1030A0006A577D4F80917D0290E08A579D4F0E9424
:1030B000D01A0E94021810E0812F0F900F900F90ED
:1030C0000F90DF91CF911F910F910895F894E82F01
:1030D000E295EF70F0E031A1282F2F7081E090E0B1
:1030E00001C0880F2A95EAF7982F9095932391A312
:1030F00092A1892B82A3789408950F931F93CF9365
:10310000DF93CBE9D1E089918F3F11F00E946618DF
:1031100081E0CF39D807B9F7C5E9D1E00BE911E073
:1031200089918F3F11F00E9466180C171D07C1F797
:10313000DF91CF911F910F910895CF92DF92EF927F
:10314000FF920F931F93CF93DF938C01C62FD0E094
:10315000CE0185569E4F7C01FC0190819F3F09F472
:1031600047C0D62EF894E92FE295EF70F0E081A1E8
:103170009F7021E030E001C0220F9A95EAF7822B80
:1031800081A382A12095282322A378940E94F51779
:10319000E5E9F1E04BE951E031E0C12C21912F3F0D
:1031A00089F0A22FA295AF70B0E090968C9190E03C
:1031B0002F7002C0959587952A95E2F780FD02C091
:1031C000832F01C080E0C82A330F4E175F0731F705
:1031D000F70180818F3F11F00E94661861E0C110F5
:1031E00001C060E08D2D0E94F717C00FD11FC8826B
:1031F000DF91CF911F910F91FF90EF90DF90CF90D3
:1032000008958091040180910401811102C094E02D
:1032100001C090E090938E0284E0891B80937D0230
:103220000E947D1888E0E6E8F2E0DF01982F1D9209
:103230009A95E9F7EEE7F2E0DF011D928A95E9F74A
:1032400084E00E9479190C943309EF92FF920F9356
:103250001F93CF93DF93CDB7DEB728970FB6F894BF
:10326000DEBF0FBECDBF8E010F5F1F4F88E0F8019C
:1032700011928A95E9F7F12C6F2DC8010E949D18D3
:10328000F394F4E0FF12F8CF48E050E0B8018EE785
:1032900092E00E94072D7C0121E0892B09F420E0B7
:1032A000E114F10441F088E0F801AEE7B2E00190EA
:1032B0000D928A95E1F760918E0270E06A577D4F1A
:1032C00044E08EE792E00E947A19EF2819F40E94F8
:1032D000041802C081E090E028960FB6F894DEBF93
:1032E0000FBECDBFDF91CF911F910F91FF90EF9057
:1032F00008950895FF920F931F93CF93DF938C014E
:10330000F62ED72FC42F222349F081E08093370275
:103310000E94612590933602809335028091370296
:103320008823C1F080913502909136020E94792560
:10333000059780F0EF2DFD2FD8014C2F50E0CD01E7
:10334000801B910B841795071CF48D918193F7CF07
:1033500010923702DF91CF911F910F91FF90089546
:10336000CF9380913A02811116C0C8EC0E94CD2CF7
:1033700081110AC08FE39CE90197F1F700C00000BA
:10338000C150A1F782E001C081E080933A0282300F
:1033900011F40E94C82C81E090913A02913009F01A
:1033A00080E0CF9108950E94B01991E08927089597
:1033B0000E94D319809304010E94B01981110C94CA
:1033C000281A08950E94B019811102C00C942A1A7B
:1033D000089581E090913B029A3008F080E00895D2
:1033E0000F931F93CF93DF93EC018B0180913B02EE
:1033F0008A3038F4B801CE010E94CE1A81111DC066
:103400000AC080913802909139020E947925843F48
:10341000914080F715C080913B028F3F19F08F5F7C
:1034200080933B0280913B028A3060F00E946125CC
:10343000909339028093380203C010923B0202C07D
:1034400080E001C081E0DF91CF911F910F9108953D
:103450000C94E72182E30C9461230F931F9398E06F
:103460008902F0011124EB5FFE4F26813781232B67
:1034700091F080938F026091060170910701209175
:10348000050130E0AB0141575D4F04E610E082E3F7
:103490000E94E82202C080E090E01F910F91089501
:1034A0005F926F927F928F929F92AF92BF92CF92D4
:1034B000DF92EF92FF920F931F93CF93DF93582EDB
:1034C00069015801C82F880FDD0B4115510531F4F2
:1034D000852D0E942D1A97FF28C025C0CE0123E01C
:1034E000880F991F2A95E1F7FC01EB5FFE4FE08002
:1034F000F12C4E155F0508F47A01FC01EB5FFE4FDD
:1035000081809280C40181579D4F3C01A7010E9498
:10351000142D04E610E09701A301682D82E30E94B8
:10352000E82297FFD5CF80E029C0A114B10429F18A
:1035300083E0CC0FDD1F8A95E1F7FE01EB5FFE4FC4
:10354000E380F12CAE14BF0408F47501CB5FDE4FAD
:103550006C817D81AB0141575D4F04E610E097011E
:1035600082E30E94152397FDDECF6C817D81615738
:103570007D4FA701C6010E94142D81E0DF91CF91FC
:103580001F910F91FF90EF90DF90CF90BF90AF9081
:103590009F908F907F906F905F9008950C94F11B97
:1035A0000C940D1C0F931F93CF93DF9300D000D08A
:1035B000CDB7DEB7609148027091490280914A020E
:1035C00090914B020E948825643671058105910512
:1035D00028F10E94A817DC01CB010296A11DB11DA4
:1035E00089839A83AB83BC8300E010E020E030E065
:1035F00044E050E0BE016F5F7F4F83E00E94501AAD
:10360000182F882361F00E946D2560934802709303
:10361000490280934A0290934B0201C011E0812F2E
:103620000F900F900F900F90DF91CF911F910F91FE
:103630000895AF92BF92CF92DF92EF92FF920F93D5
:103640001F93CF93DF937C015B016A010E94E9190C
:10365000811103C001E010E002C00AE010E0C1E007
:10366000D0E0F894B501C701F6010995789481116D
:1036700015C021960C171D0794F0CC9F9001CD9F8B
:10368000300D300D112480E090E045E34A95F1F7CC
:103690000000019682179307C1F7E3CF81E0DF9125
:1036A000CF911F910F91FF90EF90DF90CF90BF903F
:1036B000AF900895AF92BF92CF92DF92EF92FF92B8
:1036C0000F931F93CF93DF9300D000D01F92CDB7FD
:1036D000DEB75B01E0909F01F090A00101E010E0F7
:1036E0009E012B5F3F4F40E050E060E070E081E0E2
:1036F0000E94501A182F882309F43EC0670182E007
:10370000C80ED11C6091440270914502809146021E
:10371000909147020E9488256436710581059105C4
:1037200018F104E010E09E012F5F3F4F40E050E0B1
:1037300060E070E082E00E94501A182F64E070E0B0
:10374000C6010E94B91E91E02D81281390E0192333
:1037500051F10E946D25609344027093450280935D
:1037600046029093470211C064E070E0C6010E94D7
:10377000B91E9D818913D5CFF70182819381A481E0
:10378000B58189839A83AB83BC83112361F08981DE
:103790009A81AB81BC818093400290934102A093B7
:1037A0004202B09343028091400290914102A09165
:1037B0004202B0914302F50180839183A283B383D7
:1037C000812F0F900F900F900F900F90DF91CF915E
:1037D0001F910F91FF90EF90DF90CF90BF90AF902F
:1037E00008950F931F93CF93DF93EC018B014AE56C
:1037F0005BE10E94191B882351F042ED5AE1B801A8
:10380000CE01DF91CF911F910F910C94191B80E095
:10381000DF91CF911F910F9108950F931F93CF9335
:10382000DF93F894C0919F01D091A001CE01029640
:1038300024E0FB01DC0101900D922A95E1F764E0A0
:1038400070E00E94B91E89837894F8946E817F811C
:103850008885998500913C0210913D0220913E029D
:1038600030913F02601771078207930751F0609310
:103870003C0270933D0280933E0290933F020E946F
:103880008B177894DF91CF911F910F9108950E942B
:103890008E270E94F1140C949A270E949E270E9462
:1038A00089150C94B8270E94FF240E9475270E9456
:1038B000DF140E94471C0E944D1C0E94E914FBCF9C
:1038C000EF92FF920F931F93CF93DF93CDB7DEB7A5
:1038D0002C970FB6F894DEBF0FBECDBF49835A8335
:1038E0006B837C838D839E83EF82F88609871A879A
:1038F0002B873C8746E050E0BE01695F7F4FCE01D9
:1039000001960E94072D21E0892B09F420E0822FE7
:103910002C960FB6F894DEBF0FBECDBFDF91CF91CE
:103920001F910F91FF90EF9008950895E091A101EC
:10393000F091A20109950E94FD070C94951CEF924D
:10394000FF920F931F93E0904C02F0904D02009174
:103950004E0210914F02209150023091510240913D
:10396000520250915302609154027091550280911D
:103970005602909157020E94601C882321F082E534
:1039800092E00E943F24109254021092550210922D
:1039900056021092570286E0E2E5F2E0ACE4B2E0B3
:1039A00001900D928A95E1F71F910F91FF90EF9092
:1039B0000895CF93DF93CDB7DEB762970FB6F89433
:1039C000DEBF0FBECDBFE091A301F091A4014091F5
:1039D00052025091530260915402709155028091AD
:1039E0005602909157020995209352023093530248
:1039F00040935402509355026093560270935702BD
:103A000086E0E2E5F2E0DE011D9601900D928A95D6
:103A1000E1F786E0FE013D96DE01119601900D92E0
:103A20008A95E1F786E0FE013196DE011796019056
:103A30000D928A95E1F786E0FE013796A2E5B2E0A5
:103A400001900D928A95E1F74091520250915302F4
:103A500060915402709155028091560290915702E4
:103A60000E941F0820935202309353024093540245
:103A700050935502609356027093570262960FB6A8
:103A8000F894DEBF0FBECDBFDF91CF910C949F1C89
:103A9000CF93DF9300D000D000D0CDB7DEB786E063
:103AA000E2E5F2E0DE01119601900D928A95E1F7D0
:103AB00029813A814B815C816D817E8180E090E03B
:103AC00026960FB6F894DEBF0FBECDBFDF91CF9123
:103AD0000895CF93DF9300D000D000D0CDB7DEB7EC
:103AE00049835A836B837C838D839E8386E0FE01AA
:103AF0003196A2E5B2E001900D928A95E1F7269603
:103B00000FB6F894DEBF0FBECDBFDF91CF91089501
:103B1000E091A501F091A6010994CF93DF93CDB771
:103B2000DEB72C970FB6F894DEBF0FBECDBF4F8324
:103B300058878B879C870E947C1EFC0161382FEF81
:103B400072073CF09B016038710524F02FE730E0EC
:103B500001C021E8E138FF4F34F08038910524F0AE
:103B60008FE790E001C081E829878A8786E0FE011F
:103B70003796DE01119601900D928A95E1F7298121
:103B80003A814B815C816D817E8180E090E02C9652
:103B90000FB6F894DEBF0FBECDBFDF91CF91089571
:103BA00028E030E043E060E080E30C941621CF93FE
:103BB000DF93D82FC62F0E94D01D8D2F80680E94C2
:103BC0008F218C2F0E948F210E94BF218FED91E0C9
:103BD0000197F1F700C00000DF91CF910895CF93D6
:103BE000C82F0E94D01D8C2F8F770E948F210E949A
:103BF000A721C82F0E94BF218AE68A95F1F700C04D
:103C00008C2FCF9108958FE00E94EF1D28EC829FAA
:103C1000C00111240895883C910548F0893020E2C4
:103C2000920738F468EC70E00E94E12C03C068EC65
:103C300001C068E08FE00C94D71DCF93DF93209AEA
:103C40000E940E216AE58AE30E94D71D2FEF80E7CC
:103C500092E0215080409040E1F700C0000082E0F7
:103C60000E94EF1D83E00E94EF1D84E00E94EF1D83
:103C700085E00E94EF1D86E00E94EF1D62E089E36F
:103C80000E94D71D6DE183E10E94D71DEFE3FCE99F
:103C90003197F1F700C0000068E183E10E94D71D71
:103CA0000E94D01D82EE0E948F21F0E5FA95F1F777
:103CB000C8EFD1E0FE0184910E948F21F0E5FA95D2
:103CC000F1F721962DE0C63FD207A1F70E94BF2150
:103CD0008FE39CE90197F1F700C0000080E20E94A9
:103CE000EF1D682F607F80E20E94D71D80E496E080
:103CF000DF91CF910C940B1EFF920F931F93CF93E4
:103D0000DF930E94D01D80E50E948F218FE891E013
:103D10000197F1F700C000000E94A72187FF17C09C
:103D20000E94A7210E94A721082F0E94A721F82EF8
:103D30000E94A721182F0E94A721DF2D20E0C22F6B
:103D4000C02B982F88279C01212B890104C000E0FB
:103D500010E0C0E0D0E082E00E948F210E94BF21ED
:103D6000BE01C801DF91CF911F910F91FF9008957F
:103D70000895FC01680F791F8FEF91E3E617F707AD
:103D800071F02191822728E030E087FF03C0880F7F
:103D9000892701C0880F21503109B9F7EFCF089565
:103DA000CF93DF93EC01FB018281882309F43CC1AE
:103DB000C430FDE5DF0760F4CB3F9CE5D90788F40C
:103DC0009E0122503C452431310508F02EC109C026
:103DD000C236EDE5DE0729F0C63AFDE5DF0709F05A
:103DE00024C10E94161490937C0280937B02C131FF
:103DF0008CE5D80709F4C6C008F042C0C930ECE52C
:103E0000DE0709F49BC000F5C5308CE5D80709F43E
:103E100085C078F4C330ECE5DE0709F478C008F01B
:103E20007AC0C230DC4509F0F5C080917B02816028
:103E3000EFC0C7309CE5D90709F478C008F07AC014
:103E400080917B028061E4C0CD30FCE5DF0709F49E
:103E500087C058F4CB309CE5D90709F479C008F045
:103E60007BC080917B0288606FC0CF30FCE5DF07AC
:103E700009F480C008F082C080917B02877FC8C0AF
:103E8000CE3F9CE5D90709F471C000F5C531FCE5CA
:103E9000DF0709F485C068F4C3319CE5D90709F44C
:103EA00075C008F095C00E94CB0D80917B028F7782
:103EB000AFC0CC3FFCE5DF07A9F108F054C0CB3F11
:103EC000DC4509F0A7C080917C0240C0C230EDE51E
:103ED000DE0709F489C058F4C1158DE5D80709F447
:103EE0005AC008F069C080917C0282602FC0C2363F
:103EF000EDE5DE0709F47CC0C63AFDE5DF0709F40D
:103F000081C0C330DD4509F085C080E06EC080917E
:103F10007B0282607DC080917B0216C080917B0213
:103F2000886076C080917C0282604FC080917B0265
:103F300080626EC080917B0280646AC00E94CB0D5B
:103F400080917B02806864C0846062C081603DC0F3
:103F500080917B028E7F5CC080917B028D7F58C0F8
:103F600080917B0216C080917C0218C080917C02F7
:103F70008D7F2BC080917B028F7E4AC080917B0217
:103F80008F7D46C080917B028F7B42C080917B02F7
:103F9000877F8B7F3DC080917C028D7F8E7F15C097
:103FA00080917B0282FB222720F991E0922790FBEF
:103FB00082F990FB83F92CC080917C02982F909518
:103FC00091708E7F892B90FB81F980937C0222C0B7
:103FD0000E94CB0D80917B0287FB222720F991E084
:103FE000922790FB87F914C081E00E94B11412C09F
:103FF00080917B0284FB222720F991E0922790FB9D
:1040000084F906C080917B02982F909590FB80F9EF
:1040100080937B0280917B0290917C020E94271406
:104020000E94CB0D80E001C081E0DF91CF91089527
:10403000CF93DF9386319C4541F5EB010E9420131D
:10404000982F8A812091020130910301882379F011
:104050009A7A81E009F480E080935802911102C0BD
:1040600069E201C065E3C9010E94BB240AC08091D6
:104070005802811102C069E201C065E3C9010E94D2
:10408000BD240E94621380E001C081E0DF91CF91E6
:1040900008950F931F93CF93DF93C42FD22FFC016A
:1040A00082818823C9F040935B020E94612590932E
:1040B0005A028093590280E28C0F883008F057C072
:1040C000C77081E001C0880FCA95EAF7DF91CF91F0
:1040D0001F910F910C94370B80915B02481330C0F5
:1040E0008091590290915A020E947925883C91054D
:1040F00038F510E21D0FCD17B9F080E28C0F883033
:1041000040F4C77081E001C0880FCA95EAF70E94A9
:104110003E0B183028F581E09D2F977001C0880F65
:104120009A95EAF70E94370B802F0E942E0B1830C9
:10413000F0F4D77081E001C0880FDA95EAF70AC081
:1041400080E28C0F883098F4C77081E001C0880F3E
:10415000CA95EAF7DF91CF911F910F910C943E0B16
:10416000802FDF91CF911F910F910C942E0BDF9137
:10417000CF911F910F9108950F939C01CB01243F84
:104180004CE5340731F188F4293DFCE53F07D9F0CF
:104190002A3D4CE5340779F1283D3C45A9F506E276
:1041A00021EE41EE68ED7CE52BC0263FFCE53F07A4
:1041B000E1F0A8F0273F3C4539F507E225EE46EE51
:1041C00067EF7CE51DC007E225EE45EE69ED7CE575
:1041D00017C006E221EE40EE64EF7CE511C007E275
:1041E00025EE44EE65EF7CE50BC006E221EE42EEE3
:1041F00066EF7CE505C008E221E045EE6AED7CE56E
:104200000E94492080E008C0FC018281882319F0C7
:1042100010925B0201C081E00F910895289A219AC3
:10422000229A23982B9880E58CBD089590912501C2
:104230009F3F09F072C08F3F09F46FC0611103C046
:1042400010925D0203C090E290935D02423041F013
:10425000433051F0413069F490915D02946007C0A1
:1042600090915D02986003C090915D029C60909374
:104270005D0241E050E04217530718F4440F551F08
:10428000FACF90915D0240315105F1F050F4423087
:104290005105B1F048305105E1F421E020935C0272
:1042A00013C04034510591F04038510539F0403287
:1042B000510579F421E020935C0208C0936007C0A7
:1042C00091E090935C0205C0916001C09260909370
:1042D0005D022CB590915D02922B9CBD90915C0289
:1042E000992319F09DB591609DBD80932501E82F1C
:1042F000E295EF70F0E031A1282F2F7081E090E07F
:1043000001C0880F2A95EAF7932F982B91A392A1C9
:104310008095892382A381E0089580E00895CF935A
:10432000DF938EBD0E946125EC010DB407FC0AC02D
:104330000E9461258C1B9D0B84369105B0F38EEF96
:104340009FEF02C08EB590E0DF91CF910895CF939B
:10435000DF931EBC0E946125EC010DB407FC0AC06E
:104360000E9461258C1B9D0B84369105B0F38EEF66
:104370009FEF02C08EB590E0DF91CF9108958091BC
:1043800025018F3F19F1E82FE295EF70F0E031A1A0
:10439000282F2F7081E090E001C0880F2A95EAF75E
:1043A000932F982B91A392A1892B82A38FEF8093B7
:1043B00025018DB58E7F8DBD9CB580915D02809568
:1043C00089238CBD10925D0210925C0208951092B8
:1043D000B90088E48093B80008959F92AF92BF928D
:1043E000CF92DF92EF92FF920F931F93CF93DF93C1
:1043F000B82EEB010E9461256C01C431D10558F043
:10440000CF3F8FEFD80759F0CE0164E170E00E94F2
:10441000E12C7B0107C0EE24E394F12C03C025E0DE
:10442000E22EF12C84E8A82E94EA992E1092BC007A
:104430009092BC000E9461258C018091BC0087FD98
:1044400008C00E946125801B910B8E159F05A8F363
:104450002AC08091B900887F883041F08091B900EE
:10446000887F803119F00FEF1FEF1FC0B092BB00A3
:10447000A092BC000E9461258C018091BC0087FD48
:1044800008C00E946125801B910B8E159F05A8F323
:104490000AC08091B900887F883111F0803419F703
:1044A00000E010E00EC00EEF1FEFCF3F8FEFD807F8
:1044B00009F4BCCFC6010E9479258C179D0708F42A
:1044C000B5CFC801DF91CF911F910F91FF90EF9071
:1044D000DF90CF90BF90AF909F9008950F931F9360
:1044E000CF93DF93EB018093BB0084E88093BC0003
:1044F0000E9461258C018091BC0087FD0EC0CF3FDA
:104500008FEFD807C1F30E946125801B910B8C1798
:104510009D0788F38EEF9FEF0CC02091B900287F94
:1045200081E090E0283211F480E090E0919581954F
:104530009109DF91CF911F910F9108950F931F93D0
:10454000CF93DF93EC0184EC8093BC000E94612543
:104550008C018091BC0087FD0EC0CF3F8FEFD80744
:10456000C1F30E946125801B910B8C179D0788F376
:104570008EEF9FEF03C08091BB0090E0DF91CF9161
:104580001F910F9108950F931F93CF93DF93EC0129
:1045900084E88093BC000E9461258C018091BC005E
:1045A00087FD0EC0CF3F8FEFD807C1F30E94612572
:1045B000801B910B8C179D0788F38EEF9FEF03C034
:1045C0008091BB0090E0DF91CF911F910F910895F2
:1045D000CF92DF92EF92FF920F931F93CF93DF93CF
:1045E000C62F6A017901B8010E94ED2197FD11C023
:1045F000B8018C2F0E946E22E601EC0CFD1CCE153A
:10460000DF0539F097FD05C0B80189910E946E223F
:10461000F6CF24E92093BC00DF91CF911F910F9139
:10462000FF90EF90DF90CF900895CF92DF92EF92BE
:10463000FF920F931F93CF93DF93D82EC62E7A014C
:10464000E901B8010E94ED2197FD2AC0B8018C2D27
:104650000E946E2297FD24C0B8018D2D81600E94BA
:10466000ED216701219796012E193F092C173D076F
:1046700068F497FD15C0C8010E949E2297FD02C0F4
:10468000F6018083FFEFCF1ADF0AEDCF97FD08C058
:10469000C8010E94C32297FD03C0CE0DDF1D888391
:1046A00024E92093BC001816190614F480E090E069
:1046B000DF91CF911F910F91FF90EF90DF90CF90FE
:1046C00008958093BA0085EC8093BC0008951F92F2
:1046D0000F920FB60F9211242F933F934F935F9336
:1046E0006F937F938F939F93AF93BF93CF93DF93FA
:1046F000EF93FF938091B900887F803899F058F448
:10470000882309F474C0803609F073C010925E02E9
:10471000109260026EC0883A09F45BC0883B09F4CD
:1047200058C067C080915E0281111EC08091BB009D
:1047300080935F0280915F028A3020F010925F02C6
:1047400080E001C081E091E090935E0220915F02E1
:1047500030E040910601509107014217530709F0DC
:1047600090E09093600246C0E0915F02F0E080919B
:10477000BB00E157FD4F808380915F028F5F809384
:104780005F02809160028823A1F1C0919F01D091C6
:10479000A001A88188E0A802D0011124AB5FBE4F20
:1047A0001696ED91FC911797309719F114962D916B
:1047B0003C9115972C0F3D1F11968D919C9112974E
:1047C000BE01680F791F13964C9113978C91099530
:1047D00010C0E0915F02F0E0E157FD4F80818093CF
:1047E000BB0080915F028F5F80935F0202C01092D6
:1047F000BC0081E09091BC008295880F880F807C7E
:104800009568892B8093BC00FF91EF91DF91CF9148
:10481000BF91AF919F918F917F916F915F914F91D8
:104820003F912F910F900FBE0F901F90189590936E
:10483000AB018093AA01089590936702809366026A
:1048400008950E94B019811103C0809161020895FA
:10485000E0916602F0916702309721F00190F081BB
:10486000E02D099480E00895E0916602F0916702DE
:10487000309721F00280F381E02D09940895E091B2
:104880006602F0916702309739F022E0DC012C9348
:104890000480F581E02D09940895209164023091FF
:1048A00065022817390771F09093650280936402BE
:1048B000E0916602F0916702309721F00680F7815F
:1048C000E02D099408952091620230916302281727
:1048D000390771F09093630280936202E09166025F
:1048E000F0916702309721F00084F185E02D099462
:1048F0000895FC01329697E080E0915029F02191D3
:104900002223D9F38F5FF9CF0895662349F0FC0184
:10491000329608962191621729F0E817F907D1F726
:1049200080E0089581E008959C01FC0132969FEF9C
:1049300080E04191461789F09F3F19F4411101C071
:10494000982F8F5F8630A9F79F3F39F0F901E90F63
:10495000F11D97FDFA956283089508959C012A5FE1
:104960003F4FFC014281461301C01282019682171B
:104970009307B9F708950C9494240C94AE240296EE
:1049800026E0FC0111922A95E9F7089508950C9408
:10499000C62483E0809368020C94C724811102C06E
:1049A00081E001C082E0809368020C94C7240C94DB
:1049B000CE2481E0809368020C94C7240C94D924FF
:1049C00008950C94E0240C94E1240C94E0240C94BD
:1049D000E0240C94E024CF930E94E7240E94251940
:1049E0000E94E524C0E08C2F0E94EA17811104C0C8
:1049F000CF5FC830C1F701C081E0CF91089508951D
:104A00001F920F920FB60F9211248F939F93AF9323
:104A1000BF9380916902811113C080919902909196
:104A20009A02A0919B02B0919C024196A11DB11DDA
:104A30008093990290939A02A0939B02B0939C0258
:104A4000BF91AF919F918F910F900FBE0F901F90CC
:104A500018958091A102843031F10E949909109239
:104A6000690220E488E190E00FB6F894A89580935D
:104A700060000FBE2093600083B7817F846083BF96
:104A800083B7816083BF7894889583B78E7F83BF17
:104A90000FB6F894A89580916000886180936000BB
:104AA000109260000FBE08950E94CB0D0C949F09D8
:104AB00082E084BD93E095BD9AEF97BD80936E0030
:104AC00008952FB7F8948091990290919A02A0913D
:104AD0009B02B0919C022FBF08952FB7F89460916C
:104AE000990270919A0280919B0290919C022FBF33
:104AF00008959C014FB7F8948091990290919A0281
:104B0000A0919B02B0919C024FBF821B930B089512
:104B1000CF92DF92EF92FF922FB7F894C090990254
:104B2000D0909A02E0909B02F0909C022FBFA701C8
:104B30009601261B370B480B590BCA01B901FF9090
:104B4000EF90DF90CF90089578941F920F920FB658
:104B50000F9211248F939F93AF93BF9380919902EB
:104B600090919A02A0919B02B0919C020196A11D86
:104B7000B11D8093990290939A02A0939B02B093E7
:104B80009C02BF91AF919F918F910F900FBE0F909C
:104B90001F901895F89481E08093E00080E2809364
:104BA000D800E9ECF0E010828FE19EE40197F1F784
:104BB00000C000001DBA109268001CBC10BE1FBAD5
:104BC00010927A0010926E0010926F001092710095
:104BD000109272001082ECEBF0E0108214B817B85B
:104BE0001AB81DB810BA108215B818B81BB81EB87C
:104BF00011BA0C94003F08958091750208950895AC
:104C000022E02093E9002FEF3091E800215035FD9C
:104C100006C035ED3A95F1F700002111F5CF20914E
:104C2000E80025FF0BC040E050E066E070E00E9425
:104C30002A288091E8008E778093E8000895CF932A
:104C4000DF9321E02093E9002FEF3091E80021501D
:104C500035FD06C035ED3A95F1F700002111F5CF8D
:104C60002091E80025FF14C0EC0140E050E068E02E
:104C700070E00E942A288091E8008E778093E800F7
:104C800088E0FE01ADE6B2E001900D928A95E1F771
:104C9000DF91CF91089580936A0270936C026093C4
:104CA0006B028091A102843001F582E08093E900DB
:104CB0008FEF9091E800815095FD06C095ED9A9593
:104CC000F1F700008111F5CF8091E80085FF0DC05C
:104CD00040E050E063E070E08AE692E00E942A281B
:104CE0008091E8008E778093E8000895BC0184E00D
:104CF0000C944B26BC0183E00C944B268091A002BF
:104D0000811109C00E94BB290E94182A8091E200EB
:104D100084608093E20008951092A00208950C949C
:104D2000DE2460919D0281E0611101C080E00C945D
:104D3000C9249091A10281E0943009F080E0609153
:104D40009D020C94CE2442E061EC81E00E94342963
:104D500042E261EC82E00E9434299091A10281E05C
:104D6000943009F080E060919D020C94D7248091EA
:104D7000A302833009F461C030F4813071F08230D5
:104D800009F49AC008958A3009F486C08B3009F47A
:104D90006CC0893009F0A8C020C08091A202813A7D
:104DA00009F0A2C08091E800877F8093E80080919D
:104DB000A6029091A702892B21F468E08DE692E08B
:104DC00003C060E080E090E070E00E947528809170
:104DD000E8008B778093E80008958091A2028132E9
:104DE00009F082C08091A6029091A702029708F074
:104DF0007BC08091E800877F8093E8008091E80085
:104E000082FD05C08091A1028111F8CF6DC0209173
:104E1000F3008091F20090E0922B029731F48091A0
:104E2000F100813011F0863021F48091F1008093FF
:104E300075028091E8008B7753C08091A202813A7D
:104E400009F052C08091A6029091A702892B09F027
:104E50004BC08091E800877F8093E8008091E80054
:104E600080FFFCCF8091320136C08091A202813256
:104E7000D9F58091A6029091A702892BA9F580917E
:104E8000E800877F8093E8000E9469298091A4024E
:104E9000809332010C94CB0D8091A202813221F5D6
:104EA0008091E800877F8093E8000E9469298091C3
:104EB000A5028093760208958091A202813AA1F41E
:104EC0008091E800877F8093E8008091E80080FF70
:104ED000FCCF809176028093F1008091E8008E777C
:104EE0008093E8000C946929089584B7877F84BF74
:104EF0000FB6F894A8958091600088618093600057
:104F0000109260000FBE90E080E80FB6F894809396
:104F10006100909361000FBE0C94D9240E94BB29BC
:104F20000E94182AE2EEF0E0808184608083789409
:104F30000C94AD2C86E291E00C941C248091A1028B
:104F40008530A9F48091A102853079F40E94292549
:104F500080919F028823B1F30E94EB24882391F370
:104F60000E9414280E94CB0DEDCF0C945425089577
:104F700008950C94BB27292F332723303105C9F01E
:104F800060F42130310581F02230310509F044C050
:104F90008BE390E020E33EE043C021323105E1F0B5
:104FA0002232310549F138C082E190E02BE63EE043
:104FB00037C099278130910549F028F0029761F5B3
:104FC000E6EFFDE005C0ECE2FEE002C0E8E0FEE056
:104FD000849190E09F0124C06115710541F061301A
:104FE0007105D1F489E090E02BE53EE019C089E03D
:104FF00090E022E43EE014C06115710541F061309B
:10500000710551F48BE790E02DE73EE009C080E4A4
:1050100090E028EF3EE004C080E090E020E030E047
:10502000FA0131832083089580E189BD82E189BD41
:1050300009B400FEFDCF8091D8008F7D8093D80009
:105040008091E00082608093E0008091E00081FD2B
:10505000FCCF0895CF92DF92EF92FF920F931F93B0
:10506000CF93DF93EC018B017A010E948829811193
:1050700033C0E114F10439F0F70180819181081BFC
:10508000190BC80FD91FC12CD12C0115110519F10D
:105090008091E80085FD16C08091E8008E778093AE
:1050A000E800E114F10449F0F70180819181C80E14
:1050B000D91ED182C08285E00FC00E948829882332
:1050C00021F30AC089918093F10001501109FFEF8B
:1050D000CF1ADF0ADACF80E0DF91CF911F910F91D5
:1050E000FF90EF90DF90CF9008952091A80230912B
:1050F000A9022617370748F06115710539F4209188
:10510000E8002E772093E80001C0B901FC0120E0FF
:105110006115710579F18091A1028823F1F1853043
:10512000F1F18091E80083FD3CC08091E80082FDB0
:105130002EC08091E80080FFEBCF2091F30080919A
:10514000F20090E0922B6115710551F088309105C5
:1051500038F421912093F100615071090196F3CF49
:1051600021E0089709F020E08091E8008E77809395
:10517000E800CECF2111CFCF0AC08091A1028823B1
:1051800061F0853061F08091E80083FD0AC0809174
:10519000E80082FFF2CF80E0089582E0089583E086
:1051A000089581E008952091A8023091A902261760
:1051B000370748F06115710539F42091E8002E7722
:1051C0002093E80001C0B901FC0120E061157105E0
:1051D00091F18091A102882309F440C0853009F43F
:1051E0003FC08091E80083FD3DC08091E80082FDD2
:1051F0002FC08091E80080FFE9CF2091F3008091DB
:10520000F20090E0922B6115710559F088309105FC
:1052100040F424912093F100319661507109019678
:10522000F2CF21E0089709F020E08091E8008E7726
:105230008093E800CBCF2111CCCF0AC08091A1028E
:10524000882361F0853061F08091E80083FD0AC019
:105250008091E80082FFF2CF80E0089582E0089517
:1052600083E0089581E00895982F973068F5909332
:10527000E900981739F07091EC002091ED00509101
:10528000F00003C0242F762F50E021FD02C09F5F65
:10529000ECCF3091EB003E7F3093EB003091ED008E
:1052A0003D7F3093ED003091EB0031603093EB00A7
:1052B0007093EC002093ED005093F0002091EE00ED
:1052C00027FDE5CF80E008958F708093E90081E0AD
:1052D00008958091A20287FF11C08091E80082FDAD
:1052E00005C08091A1028111F8CF11C08091E80022
:1052F0008B770BC08091A102882349F08091E80050
:1053000080FFF8CF8091E8008E778093E8000895C1
:105310002091E4003091E50095E64091EC00842F67
:10532000817040FF23C08091E80080FD1DC0809106
:10533000A102882399F0853099F08091EB0085FDDA
:1053400011C04091E4005091E5002417350729F37E
:10535000915011F09A01E1CF84E0089582E0089520
:1053600083E0089581E0089580E008954091E80089
:1053700042FFDDCF08950E94292A0E94312AE0EEE3
:10538000F0E0808181608083E8EDF0E080818F77BC
:10539000808319BCA7EDB0E08C918E7F8C938081C7
:1053A0008F7E80831092A00208950F931F93CF9356
:1053B000DF930E94292A0E94312AC8EDD0E088811B
:1053C0008F77888388818068888388818F7D8883B0
:1053D00019BC1092A10210929D0210929F0210928D
:1053E0009E0200EE10E0F80180818B7F808388812F
:1053F0008160888342E060E080E00E943429E1EE31
:10540000F0E080818E7F8083E2EEF0E08081816039
:105410008083808188608083F80180818E7F808393
:10542000888180618883DF91CF911F910F910895CA
:10543000E8EDF0E080818F7E8083E7EDF0E0808111
:105440008160808384E082BF81E08093A0020C941D
:10545000D529E8EDF0E080818E7F80831092E20014
:1054600008951092DA001092E10008951F920F92B1
:105470000FB60F9211242F933F934F935F936F9327
:105480007F938F939F93AF93BF93EF93FF938091FD
:10549000E10082FF0BC08091E20082FF07C0809193
:1054A000E1008B7F8093E1000E94AC2C8091DA00B8
:1054B00080FF1FC08091D80080FF1BC08091DA0060
:1054C0008E7F8093DA008091D90080FF0DC080E14B
:1054D00089BD82E189BD09B400FEFDCF81E08093E2
:1054E000A1020E947E2605C019BC1092A1020E9452
:1054F0008C268091E10080FF19C08091E20080FF3E
:1055000015C08091E2008E7F8093E2008091E200DE
:1055100080618093E2008091D80080628093D800FF
:1055200019BC85E08093A1020E9491268091E10040
:1055300084FF30C08091E20084FF2CC080E189BDEF
:1055400082E189BD09B400FEFDCF8091D8008F7D36
:105550008093D8008091E1008F7E8093E10080915C
:10556000E2008F7E8093E2008091E2008160809370
:10557000E20080919D02882311F084E007C08091B1
:10558000E30087FD02C081E001C083E08093A102B7
:105590000E9499268091E10083FF29C08091E2005A
:1055A00083FF25C08091E100877F8093E10082E046
:1055B0008093A10210929D028091E1008E7F8093E2
:1055C000E1008091E2008E7F8093E2008091E20012
:1055D00080618093E20042E060E080E00E94342934
:1055E0008091F00088608093F0000E948F26FF91E8
:1055F000EF91BF91AF919F918F917F916F915F914B
:105600004F913F912F910F900FBE0F901F901895C3
:105610001F920F920FB60F9211242F933F934F9327
:105620005F936F937F938F939F93AF93BF93CF932A
:10563000DF93EF93FF93C091E900CF708091EC006E
:10564000D82FD17080FDD0E81092E9008091F00051
:10565000877F8093F00078940E944C2B1092E90091
:105660008091F00088608093F000CD2BCF70C093C4
:10567000E900FF91EF91DF91CF91BF91AF919F91A1
:105680008F917F916F915F914F913F912F910F90EB
:105690000FBE0F901F9018951F93CF93DF93CDB738
:1056A000DEB7AA970FB6F894DEBF0FBECDBFE2EA11
:1056B000F2E08091F100819322E0EA3AF207C9F723
:1056C0000E94B7268091E80083FF2EC18091A2023C
:1056D0009091A302492F50E04A30510508F024C1AF
:1056E000FA01EE59FF4F0C94F52C803821F08238E6
:1056F00009F01AC108C080919E0290919F029923DF
:1057000089F082600FC08091A6028F70873008F008
:105710000BC18093E9008091EB0085FB882780F91D
:105720001092E9009091E800977F9093E8008093B1
:10573000F1001092F100D1C0282F2D7F09F0F4C0A4
:10574000882319F0823061F0EFC08091A40281308B
:1057500009F0EAC0933009F080E080939F022EC0E8
:105760008091A40281112AC08091A6028F702FEF30
:10577000280F263008F0D8C08093E9002091EB0074
:1057800020FF1CC0933021F48091EB00806214C094
:105790009091EB0090619093EB0021E030E0A90143
:1057A00002C0440F551F8A95E2F74093EA00109219
:1057B000EA008091EB0088608093EB001092E90092
:1057C0008091E800877F8093E8000E946929ACC03F
:1057D0008111AAC01091A4021F778091E300807804
:1057E000812B8093E3008091E800877F8093E8001D
:1057F0000E9469298091E80080FFFCCF8091E3003E
:1058000080688093E300111102C082E001C083E050
:105810008093A10289C08058823008F085C08091B1
:10582000A4029091A5028C3D53E0950779F583E0A1
:105830008A838AE289834FB7F894DE01139620E0C9
:105840003EE051E2E32FF0E050935700E49120FF57
:1058500003C0E295EF703F5FEF708E2F90E0EA306B
:1058600010F0C79601C0C0968D939D932F5F243191
:1058700049F74FBF8091E800877F8093E8006AE294
:1058800070E0CE0101960E94752816C06091A602B4
:105890007091A702AE014F5F5F4F0E94B927BC0114
:1058A000892B09F441C09091E800977F9093E8001C
:1058B00089819A810E94D3288091E8008B77809318
:1058C000E80032C0803881F58091E800877F8093BE
:1058D000E80080919D028093F1008091E8008E772E
:1058E00072CF811121C08091A4029091A5029927C5
:1058F0000297D4F48091E800877F8093E80080913C
:10590000A40280939D020E94692980919D028111C9
:1059100006C08091E30087FD02C081E001C084E001
:105920008093A1020E94A3268091E80083FF0AC011
:105930008091E800877F8093E8008091EB0080628F
:105940008093EB00AA960FB6F894DEBF0FBECDBFD2
:10595000DF91CF911F9108950895CF938091A10277
:105960008823A1F0C091E900CF709091EC00892FBD
:10597000817090FD80E8C82B1092E9008091E800CA
:1059800083FD0E944C2BCF70C093E900CF91089506
:105990000E94BB291092A10208958091E300881F04
:1059A0008827881F089587FB082E062687FD819586
:1059B00067FD61950E94FB2C0EF4919507FC819583
:1059C0000895AA1BBB1B51E107C0AA1FBB1FA61746
:1059D000B70710F0A61BB70B881F991F5A95A9F798
:1059E00080959095BC01CD010895EE0FFF1F0590A5
:1059F000F491E02D0994991B79E004C0991F961742
:105A000008F0961B881F7A95C9F780950895FB01C9
:105A1000DC0104C08D910190801921F44150504067
:105A2000C8F7881B990B0895FB01DC0102C00190A7
:105A30000D9241505040D8F70895F999FECF92BD8C
:105A400081BDF89A992780B50895A6E1B0E044E0B9
:105A500050E00C94572DA8E1B0E042E050E00C94E7
:105A6000572D262FF999FECF92BD81BDF89A019747
:105A700000B4021639F01FBA20BD0FB6F894FA9A96
:105A8000F99A0FBE08950396272F0E94322D0E9487
:105A9000312D252F0E94322D242F0C94322D01966A
:105AA000272F0E94322D0C94312DDC01CB01FC01FB
:105AB000F999FECF06C0F2BDE1BDF89A319600B467
:0E5AC0000D9241505040B8F70895F894FFCF72
:105ACE00C8001902010100000000000000000000E3
:105ADE0001010000000000000402000000040600A6
:105AEE000000000000FFFC251F2600267A267626E1
:105AFE00FF2501E200E900EA00B500B600B700CDCF
:105B0E00008301CC008A0192019401210223022418
:105B1E00022502260227022A02B300B4006F00708B
:105B2E0000818283E200E900EA00B500B600B7000A
:105B3E00CD008301CC008A0192019401210223023F
:105B4E0024022502260227022A02B300B4006F00A7
:105B5E007000818283969734936667F63536F78F99
:0A5B6E00021D1E8D1D0B1E031E00FC
:00000001FF
